:100000008A010228831287011B3083168700803003
:1000100094000E3093002830831294008C118316C4
:1000200011148316111C1528112883128C1190307D
:10003000930083120C080839003C0130031D0301B2
:10004000003C03192428192883128C114030930096
:1000500083120C080839003C0130031D0301003CE9
:100060000319332828288312A00183128C11200839
:10007000930083120C080839003C0130031D030172
:0E008000003C0319442839288312A00A3528B1
:00000001FF
